:103E71000F580F4E0F430F380F2D0F210F140F073F
:103E81000EF90EEB0EDC0ECC0EBC0EAB0E9A0E87AD
:103E91000E750E610E4D0E380E220E0C0DF40DDC5A
:103EA1000DC40DAA0D900D750D5A0D3E0D210D037A
:103EB1000CE40CC50CA50C850C640C420C200BFD0C
:103EC1000BD90BB50B900B6B0B460B200AF90AD3E0
:103ED1000AAC0A840A5D0A350A0D09E409BC099392
:103EE100096B0942091A08F108C808A008780850A6
:103EF1000828080007D807B1078A0764073E071892
:103F010006F206CD06A906840661063E061B05F8E3
:103F110005D705B50595057405550535051704F94A
:103F210004DB04BE04A20486046A044F0435041BA6
:103F3100040203E903D103B903A2038B0375035FF1
:103F4100034A03350321030D02FA02E702D502C336
:103F510002B102A0028F027F026F025F0250024192
:103F6100023302250217020A01FD01F001E301D724
:103F710001CC01C001B501AA019F0195018B01810D
:103F81000178016E0165015C0154014B0143013B64
:103F91000133012C0125011D011601100109010246
:103FA10000FC00F600F000EA00E500DF00DA00D4D2
:103FB10000CF00CA00C600C100BC00B800B300AF0A
:103FC10000AB00A700A3009F009B00980094009104
:103FD100008D008A00870084008100010C01010529
:103FE10002011E030A960401320503030600640759
:103FF100010108000009015A0E01010F0001120020
:104001006413010114013C1501FA1664FA17FFFF4C
:104011001D00072000072400022701012F013C3069
:10402100030332010335FFFF3603073CFFFF3DFF6A
:10403100FF180002191E461A00021B00022D32C889
:064041002E0001FAFAFA5C
:10004800900786E0FEA3E0FF7457BE0010D39F40E0
:100058000C903FDB12001EE493F5998012900786FE
:10006800E0FEA3E0FF903FDB12001EE493F59990B9
:10007800078612000E900786E0FEA3E0FF746C6FFF
:100088004E700375130022900072E0B402087401E8
:10009800900072F0D20E90013AE090002AF09001A0
:1000A8003BE090002BF090013CE090002CF0A20A7D
:1000B800B3401690013AE0700C90013BE070069056
:1000C800013CE060028002C20A90013AE0B4300FBD
:1000D80090013BE0B4470890013CE0643B6002803B
:1000E80004D20B8002C20BE559B40102800302025C
:1000F80011900057E0F567900062E0F569900063A1
:10010800E0F56A900074E0F56B90007AE0900029C1
:10011800F090007CE0F56690007DE0F56890008046
:10012800E0F565900081E0F564900090E090004172
:10013800F0900091E0900042F0900092E09000432F
:10014800F0900093E0900044F0900094E090004517
:10015800F0900095E0900046F0900096E0900047FF
:10016800F0900097E0900048F0900099E0900033FC
:10017800F090009AE0900034F090009BE0900035F9
:10018800F090009CE0900036F0900079E0B4011700
:1001980090000A740FF0A374FFF090000CE4F0A331
:1001A800F07402900079F0900079E0B4035990005F
:1001B8000CE0FEA3E0FF90000AE0FCA3E0FD1200C3
:1001C8000374101241A77408124199EF900026F0A9
:1001D800EF700674FF900026F07400900079F0909C
:1001E800000BE0900027F090000AE0900028F090C3
:1001F8000026E0900789F0900027E090078AF090A9
:100208000028E090078BF0803F900081E070067531
:100218005901756400A20AB3402E90013AE090009B
:100228002AF090013BE090002BF090013CE0900018
:100238002CF090002AE0700C90002BE070069000E3
:100248002CE060028002C20AE5677003756702E568
:100258006970037569027E837FC2E5678E048F0526
:10026800FF1241898C398D3AE56A75F0FAA4FFAE20
:10027800F0E5698E048F05FF1241898C3D8D3E9013
:10028800004FE0F56190004DE0FE900069E0B50692
:100298001890004CE0FE900068E0B5060C90004B0A
:1002A800E0FE900059E06E606F900069E070069083
:1002B8000068E060067400900059F0900069E0B4AE
:1002C80002089000497401F08005900049E4F0901C
:1002D8000068E0B4020890004A7401F080059000BC
:1002E8004AE4F0900068E0600690004AE06002800E
:1002F800057561048003756105E55AB55902D20E8A
:10030800900068E090004CF0900069E090004DF09B
:10031800900059E090004BF0740190009EF074003A
:1003280090009FF074009000A0F074009000A1F07D
:1003380074009000A2F074009000A3F07400900084
:10034800A4F074019000A5F074009000A6F0740069
:100358009000A7F074009000A8F074019000A9F034
:1003680074009000AAF074009000ABF07401900043
:10037800ACF074019000ADF074009000AEF0740021
:100388009000AFF074019000B0F074009000B1F0EC
:1003980074009000B2F07401900362F0740190034D
:1003A80063F07400900364F07400900365F07401C6
:1003B800900366F07400900367F07400900368F08F
:1003C80074019003A2F074019003A3F074009003E9
:1003D800A4F074019003A5F074019003A6F07400D2
:1003E8009003A7F074009003A8F074009003E2F063
:1003F80074019003E3F074009003E4F07401900337
:10040800E5F074009003E6F074009003E7F07400E0
:100418009003E8F07400900422F07400900423F034
:100428007400900424F07400900425F07400900483
:1004380026F07400900427F07400900428F07400EB
:10044800900462F07400900463F07401900464F006
:100458007401900465F07400900466F074009004D0
:1004680067F07400900468F022E5B554F7F5B5E537
:10047800B554FDF5B5C293C294C291C2927570008D
:10048800757100C290C207E5B554FBF5B575510505
:10049800E55104F55290004FE0F561900025E4F035
:1004A800C209E5B554FEF5B5C28E758D00758B0091
:1004B800754C00752600752500D28E22750A0075C8
:1004C8000900AE09AF0A7457BE00039F5003020526
:1004D80081903FDB12001EE49390004E1241BF0F43
:1004E800BF00010EE0FC903FDB12001EECFEE4931F
:1004F800FFEEC39F5026AE09AF0A0FBF00010E9052
:100508003FDB12001EAE09AF0AE493FC903FDB12FA
:10051800001EE49390004E1241BFECF0AE09AF0A02
:10052800903FDB12001EE49390004E1241BFE0FCA6
:10053800903FDD12001EECFCE493FDECD39D4019C6
:10054800903FDD12001EE493FC903FDB12001EE496
:100558009390004E1241BFECF0AE09AF0A74022F1F
:10056800FF50010E8E098F0A780A740126F650048E
:1005780018E436F640030204CA22750A0075090019
:10058800AE09AF0A7415BE00039F500302064F90D0
:10059800403212001EE49390004E1241BF0FBF007C
:1005A800010EE0FC90403212001EECFEE493FFEED8
:1005B800C39F5026AE09AF0A0FBF00010E9040320C
:1005C80012001EAE09AF0AE493FC90403212001EDE
:1005D800E49390004E1241BFECF0AE09AF0A904090
:1005E8003212001EE49390004E1241BFE0FC90408E
:1005F8003412001EECFCE493FDECD39D40199040AE
:100608003412001EE493FC90403212001EE49390D2
:10061800004E1241BFECF0AE09AF0A740F6F4E7076
:1006280006750A15750900AE09AF0A74022FFF5046
:10063800010E8E098F0A780A740126F6500418E410
:1006480036F6400302058822054D22054C22054E48
:10065800C2CF2290F800E4936406600280FE75849D
:100668000175A70075FF80900788E4F075C91075BB
:10067800A70F75A1C775A70075D90075CEFF75A717
:100688000F75F1FE75F2FF75F33775F47875A4BA36
:1006980075A5FF75A60775AE0075AFFF75D4817592
:1006A800D5FF75D6FF75D7FFE5B554EFF5B5E5B5B8
:1006B80054DFF5B5C287E5B554BFF5B5E5B5547F48
:1006C800F5B5E5B554F7F5B5E5B554FDF5B575A738
:1006D8000075A20175A14775F80975BC0175BE04BE
:1006E80075BD6C75BE0775BDA075BE0875BD017575
:1006F800BC0075BB1875BC2075BA0875E88075D143
:100708001375A70F75E10575E20075C74075970069
:10071800759780740A1241797597C0E597542070CF
:100728000280F8758F0275A700D2AF75980075A979
:100738000C75A70F75AB4375ADFB75AC1E75A7009F
:10074800758911758E00758C00758A00D2A9D28CB6
:10075800758D00758B00D2ABD28E75CD0075CC002F
:1007680075CA0075CB00D2ADC2CFD2CA75910475D7
:1007780092007593CD75EF0675D94075CF01900736
:1007880086E4F0A3F0751300751400C299D20AC26A
:100798000F12047174C8F5187517001227A075A7F1
:1007A8000FE5FB90001AF0E5FA90001BF0E5F990D0
:1007B800001CF075A70090F800E493F5081228D7FC
:1007C800122E11900789E0900026F090078AE09099
:1007D8000027F090078BE0900028F090078CE090BD
:1007E8000029F090078DE0F56790078EE0F5699095
:1007F800078FE0F56A900790E0F56B900791E0F5B8
:1008080066900792E0F568900793E0F56590079485
:10081800E0F564900795E090002AF0900796E09044
:10082800002BF0900797E090002CF0900798E0904C
:100838000041F0900799E0900042F090079AE0900C
:100848000043F090079BE0900044F090079CE090F4
:100858000045F090079DE0900046F090079EE090DC
:100868000047F090079FE0900048F09007A0E090C4
:100878000033F09007A1E0900034F09007A2E090D8
:100888000035F09007A3E0900036F07400900082E5
:10089800F090013AE0700C90013BE0700690013C4A
:1008A800E060028004C20A8002D20A90F807E4934A
:1008B800900021F0900021E0440A900021F090007F
:1008C80021E054FE900021F07406900012F07402AA
:1008D800900013F090F802E493900014F0740390E1
:1008E8000015F07403900016F0741D900017F07452
:1008F80005900018F07405900019F090F804E4933E
:1009080090001DF0740090001EF090F805E493909C
:10091800001FF090F806E493900020F074FF900018
:1009280022F0745A900125F07446900126F0742044
:10093800900127F07435900128F07448900129F04F
:10094800745090012AF0743190012BF074399001A1
:100958002CF0742090012DF0743590012EF0745312
:1009680090012FF07470900130F07465900131F0AF
:100978007465900132F07464900133F090007AE06D
:10098800D394014006740090007AF0755901755AA5
:1009980001740390004CF012008F1204C4120582F7
:1009A8001227CCE5B554FEF5B5900025E4F0900784
:1009B80086E4F0A3F0752400752300754800752AB5
:1009C80000752900754900753200753100754A00B7
:1009D800755400755500755B0075510575520175A4
:1009E800343C7533007573007572007574CD755697
:1009F800007557007558007543007544007545002B
:100A0800754600755C007547007542007541009099
:100A18000006E4F0A3F0900008E4F0A3F0755F008E
:100A280075600090000E74FDF0A374E8F090002348
:100A3800E4F07464900024F0C200D201C202D20330
:100A4800754D00756E00C297C2A0C296C295C2A22B
:100A5800C20E7E017F00900028E01241A790002777
:100A6800E02FFF50010E90000AEEF0A3EFF0900087
:100A780026E0700674FF900026F090000AE0FEA3BE
:100A8800E0FFEFD394FFEE940F400790000AE4F0E4
:100A9800A3F07400900071F07400900079F0740075
:100AA800900082F0740090008DF074009000B4F013
:100AB800E5687003756804743A90074EF074FD9009
:100AC800074FF0900414E0900454F0D2B0D2B7D29B
:100AD800A7D2A6D2B1D2A3C207A2B6B39204A2B338
:100AE800B39205D29CD2EC75CF01A298B34005C24F
:100AF80098123175E5136006A299B3B340028005D8
:100B0800C2991236E5E51464016005E514B40402DF
:100B180080D5E54DD39405400CE55BC394C85002DD
:100B2800055B754D00E574C394F0501A7872120095
:100B38003FAE72AF73EFD394E8EE940340080574A8
:100B4800757300757200C28E7E047F00E54C1241F9
:100B5800A7E58D75F004A4FDACF0EF2DFDEE3CFC8F
:100B6800E58B75F04084FF7E00ED2FFFEC3EFE8E96
:100B7800258F26D28EA2B6300401B35003020CC2D0
:100B8800A2B6300401B35003020CC2A2B6406705F6
:100B980054A20F400575FFA0D20FE5B54401F5B585
:100BA800900024E4F0E554D3956740487C837DC2E7
:100BB800AE25AF261240478E238F24E5482FFF50DD
:100BC800010E74011241998E238F2485244875548F
:100BD80001C28E758D00758B00754C00D28E740322
:100BE800BE00039F50069000257401F0E543B4064B
:100BF80003754300D204A2B6B35003020CC2C20468
:100C080090006BE06018123826A200B34008E5B5E2
:100C18004408F5B58006E5B554F7F5B58002C2007D
:100C280090006EE0601812397BA202B34008E5B567
:100C38004402F5B58006E5B554FDF5B58006E5B581
:100C480054FDF5B5A207B34004D2968002C296902F
:100C58000059E06004D2958002C29590004AE0B441
:100C68000104D2978002C297900049E0B40104D2EF
:100C7800A08002C2A0A209B34004D2A28002C2A2EC
:100C8800900018E0FE900014E0C39E400990001404
:100C9800E0D39408400974FB900023F0120471908B
:100CA800001DE0601590001DE0FE900017E06E60EA
:100CB8000974FE900023F0120471C2CA7E017F00FD
:100CC800E54E1241A7E5CD2FFF50010E8E278F2844
:100CD800D2CAE566B4014890000EE0FCA3E0FDEF3F
:100CE800C39DEE9C4039B208E52A45296013A20845
:100CF800B34008E5B54404F5B58006E5B554FBF501
:100D0800B590000EE0FEA3E0FF900010E0FCA3E029
:100D1800FDEF2DFDEE3CFC90000EECF0A3EDF0A2F3
:100D2800B3300501B35003020E10A2B3300501B36E
:100D38005003020E10A2B35003020E090555A20F6C
:100D4800400575FFA0D20FE5B54401F5B590002424
:100D5800E4F0E555D395695003020E077CEA7D60FF
:100D6800AE27AF281240478E298F2AE56A1241A77D
:100D780074FF8E048F05FF1241898C298D2AE5495D
:100D88002DFD50010C74018C068D071241998E2996
:100D98008F2A852A49A209B3401574641241A79085
:100DA8000067E08E048F05FF1241898C298D2A7512
:100DB800550190000EE0FEA3E0FFAC27AD2812001D
:100DC8000390000EEEF0A3EFF0E568FF124189747E
:100DD8000AFF12418990007BE08C068D071241A71B
:100DE80074148E048F05FF124189900010ECF0A353
:100DF800EDF0C2CA75CD0075CC00754E00D2CAD2CE
:100E080005A2B3B34002C205900025E0B40107E58E
:100E180056C394064003021424E56E90277FF828F1
:100E28002873900059E0C394024003020F7EE551F5
:100E3800D394015003020F7EE55175F040A4FFAE34
:100E4800F090031212001EE0C395455018E5517545
:100E5800F040A4FFAEF090031112001EE0F52E75CD
:100E68002D00020F7EE55175F040A4FFAEF090030F
:100E78001012001EE0C395454003020F1AE5517594
:100E8800F040A4FFAEF090031112001EE55175F07A
:100E980040A4FFAEF0E0FC90030F12001EECFEE051
:100EA800FFEEC39FFEE5518E0475F040A4FFAEF03F
:100EB80090031012001EE0F40425458C0088F0A46D
:100EC800FFAEF0E5518F048E0575F040A4FFAEF03B
:100ED80090031212001EE55175F040A4FFAEF0E039
:100EE800FA90031012001EEAFEE0FFEEC39FFECD4B
:100EF800CCCD8E07124189E55175F040A4FFAEF0C4
:100F080090030F12001EE02DFD50010C8C2D8D2E2C
:100F18008064E55175F040A4FFAEF090030F120015
:100F28001EE55175F040A4FFAEF0E0FC90030E12F0
:100F3800001EECFEE0FFEEC39F8545F0A4FFAEF077
:100F4800E5518F048E0575F040A4FFAEF0900310B4
:100F580012001EE0FECDCCCD8E07124189E55175F9
:100F6800F040A4FFAEF090030E12001EE02DFD50DD
:100F7800010C8C2D8D2E756E01021424900059E001
:100F8800C39402400302113290004FE0D3955150B0
:100F9800030210DAE55175F040A4FFAEF090031893
:100FA80012001EE0C395455018E55175F040A4FFA6
:100FB800AEF090031712001EE0F52C752B000210FE
:100FC800DAE55175F040A4FFAEF090031612001E4A
:100FD800E0C395454003021076E55175F040A4FF43
:100FE800AEF090031712001EE55175F040A4FFAE55
:100FF800F0E0FC90031512001EECFEE0FFEEC39F2C
:10100800FEE5518E0475F040A4FFAEF09003161271
:10101800001EE0F40425458C0088F0A4FFAEF0E53E
:10102800518F048E0575F040A4FFAEF0900318129E
:10103800001EE55175F040A4FFAEF0E0FA900316EB
:1010480012001EEAFEE0FFEEC39FFECDCCCD8E0758
:10105800124189E55175F040A4FFAEF090031512D6
:10106800001EE02DFD50010C8C2B8D2C8064E55169
:1010780075F040A4FFAEF090031512001EE55175FF
:10108800F040A4FFAEF0E0FC90031412001EECFE4A
:10109800E0FFEEC39F8545F0A4FFAEF0E5518F0455
:1010A8008E0575F040A4FFAEF090031612001EE006
:1010B800FECDCCCD8E07124189E55175F040A4FFD5
:1010C800AEF090031412001EE02DFD50010C8C2B85
:1010D8008D2CE551B40123E561D39401401CE556FC
:1010E80004D395514014E545C39405500D90035F12
:1010F800E0A829B80006952A40028003755102E548
:1011080051B5612290004FE0D395514019E55175D2
:10111800F040A4FFAEF090031712001EE0A823B819
:1011280000069524400280020561756E02021424AF
:10113800900059E0B4022AE55175F040A4FFAEF0E2
:1011480090031712001EE0F52C752B00E55175F081
:1011580040A4FFAEF090030E12001EE0F52E752D90
:1011680000900059E0B4030F900051E0F52C752B66
:1011780000752E00752D00756E03021424E5517557
:10118800F040A4FFAEF090032012001EE0C3955B70
:10119800400302125A900049E07036E551D3940199
:1011A8004029AE23AF24AC2DAD2EEDD39FEC9E404D
:1011B8001AE55175F040A4FFAEF090031E12001E10
:1011C800E0A829B80005D3952A500280021551805D
:1011D80034E551D394024029AE23AF24AC2DAD2E73
:1011E800EDD39FEC9E401AE55175F040A4FFAEF098
:1011F80090031E12001EE0A829B80005D3952A50B6
:101208000280021551E551B55237E551C395615039
:1012180030E55604D395514028AE23AF24AC2BAD0E
:101228002CEFD39DEE9C4019E55175F040A4FFAE1C
:10123800F090031F12001EE0A829B80006952A4066
:101248000280020551C290E55165526005C20775DA
:101258005B00756E04021424E55175F040A4FFAEDE
:10126800F090031A12001EE0B40117E55175F04022
:10127800A4FFAEF090032012001EE0240AC3955B81
:101288004003021330753064752F00A207B3500B6A
:10129800900060E02405C395454003021330E551F2
:1012A80075F040A4FFAEF090031D12001EE0C39538
:1012B800454064E55175F040A4FFAEF090031C1260
:1012C800001EE55175F040A4FFAEF0E0FC90031B52
:1012D80012001EECFEE0FFEEC39F8545F0A4FFAEB2
:1012E800F0E5518F048E0575F040A4FFAEF0900331
:1012F8001D12001EE0FECDCCCD8E07124189E551AE
:1013080075F040A4FFAEF090031B12001EE02DFD07
:1013180050010C8C2F8D30AE23AF24AC2FAD30EFA5
:10132800D39DEE9C4002D207756E05021424E55148
:10133800B40109900059E0C39402400302140490D8
:101348000358E0D395455003021404900356E0C3B4
:1013580095455040900357E0FE900355E0F4042E65
:10136800FE900356E0F40425458E0088F0A4FFAEF5
:10137800F0900358E0FC900356E0F4042C8E048FA0
:1013880005FF124189900355E02DFD50010C8C2B6F
:101398008D2C802C900355E0FE900354E0F4042E2D
:1013A8008545F0A4FFAEF0900356E08E048F05FF4C
:1013B800124189900354E02DFD50010C8C2B8D2C8B
:1013C800E551C395615030E55604D395514028AE98
:1013D80023AF24AC2BAD2CEFD39DEE9C4019E551E7
:1013E80075F040A4FFAEF090031F12001EE0A8297C
:1013F800B80006952A40028003755102900049E022
:10140800B40106E551640160028003755102E5519B
:0C14180065526005C207755B00756E0030
:10277F00020E2A020F840211380211850212600222
:02278F001336FF
:10142400900050E02402A823B80007D3952440027A
:10143400C207900025E0B40109900059E0C3940369
:1014440040030215AC900049E060030214FBE5512F
:10145400D394014034E55175F040A4FFAEF09003FD
:101464001412001EE0A823B8001FD39524401AE5E7
:101474005175F040A4FFAEF090031F12001EE0A8C7
:1014840029B80005D3952A500280021551E551D39D
:101494009401402FE55175F040A4FFAEF090031283
:1014A40012001EE0C39545501AE55175F040A4FFA3
:1014B400AEF090031E12001EE0A829B80005D395D3
:1014C4002A500280021551E551D394014022E55679
:1014D40004C39551501AE55175F040A4FFAEF09045
:1014E400031E12001EE0A829B80005D3952A500255
:1014F400800215510215A1E551D394024034E551FF
:1015040075F040A4FFAEF090031412001EE0A8236F
:10151400B8001FD39524401AE55175F040A4FFAEDE
:10152400F090031F12001EE0A829B80005D3952AE5
:10153400500280021551E551D39402402FE55175B4
:10154400F040A4FFAEF090031212001EE0C39545D4
:10155400501AE55175F040A4FFAEF090031E12003E
:101564001EE0A829B80005D3952A5002800215511F
:10157400E551D394024022E55604C39551501AE52F
:101584005175F040A4FFAEF090031E12001EE0A8B7
:1015940029B80005D3952A500280021551E55165FA
:1015A400526005C207755B00900060E0D39545501A
:1015B40009900054E0C395455002C207900059E0D9
:1015C4007003021811A2A5B34008A2A4B3400302F9
:1015D40017FAAE35AF367441D39F749C9E4005789C
:1015E4003512003FAE35AF36EFB48806EEB41302C1
:1015F40080030217D7A2A5500302169A900059E05F
:10160400B4010B90004FE0D3956140020561900056
:1016140059E0B40254E55175F040A4FFAEF09003D4
:101624002012001EE0C3955B503F90004FE0D3951D
:10163400514021E55604D395514019E55175F040C8
:10164400A4FFAEF090031412001EE0A823B8000615
:10165400952440028002055190004FE0F561E55168
:1016640065526005C207755B00900059E0B403261B
:1016740090004FE0D395514008E55604D39551505E
:10168400028002055190004FE0F561E5516552601A
:1016940005C207755B00A2A450030217D790005936
:1016A400E0B4016E900049E07035E551D3940140F7
:1016B40029E55175F040A4FFAEF090031E12001E00
:1016C400E0A829B8000FD3952A400A1551755B008C
:1016D400855161800385516180037561018033E523
:1016E40051D394024029E55175F040A4FFAEF09027
:1016F400031E12001EE0A829B8000FD3952A400A41
:101704001551755B008551618003855161800375B6
:101714006102900059E0D3940150030217CBE551C4
:1017240075F040A4FFAEF090032012001EE0C395B4
:101734005B40030217CB900049E07041E551D3941C
:10174400014034E55175F040A4FFAEF0900311124E
:10175400001EE0A823B8001FD39524401AE5517554
:10176400F040A4FFAEF090031E12001EE0A829B8BA
:101774000005D3952A500280021551803FE551D3CC
:1017840094024034E55175F040A4FFAEF09003118B
:1017940012001EE0A823B8001FD39524401AE55177
:1017A40075F040A4FFAEF090031E12001EE0A829BD
:1017B400B80005D3952A500280021551E5516552AF
:1017C4006005C207755B00E556B40704055F800336
:1017D400755F00E564B4010EAE35AF36EF6440705A
:1017E40005EE649C6002800EA2A54003755901A217
:1017F400A44003755902A2A5B3B35006A2A4B3B37F
:10180400400280067536007535000218FFA2A5B3A4
:101814004008A2A4B340030218EBAE35AF367441BE
:10182400D39F749C9E4005783512003FAE35AF3689
:10183400EFB48806EEB4130280030218EBA2A540AD
:101844006F900068E0605A90004AE0B4010790008D
:101854004AE4F0800690004A7401F090004AE07077
:1018640005756104800375610590004AE0B40104C4
:10187400D2978002C297E551B4051AE55175F0403C
:10188400A4FFAEF090031E12001EE0A829B80005C4
:10189400D3952A50028008755104C207755B0080F5
:1018A40003756105E556B40704055F8003755F00A1
:1018B400A2A44033900069E06021900049E0B401A3
:1018C40007900049E4F080069000497401F090000C
:1018D40049E0B40104D2A08002C2A0E556B40704D2
:1018E400055F8003755F00A2A5B3B35006A2A4B33D
:1018F400B340028006753600753500E559655A60B7
:1019040006900082E06003021A87C29C7514007579
:101914001300C2CAE559902791F82828738012123F
:101924002E11800D122EEA8008122FC3800312306C
:011934009C16
:0F27910002192102192302192802192D021932E7
:10193500900029E090007AF0E567900057F0E5699E
:10194500900062F0E56A900063F0E56B900074F03A
:10195500E56690007CF0E56890007DF0E565900017
:1019650080F0E564900081F090002AE090013AF063
:1019750090002BE090013BF090002CE090013CF0B2
:10198500900041E0900090F0900042E0900091F0CE
:10199500900043E0900092F0900044E0900093F0B6
:1019A500900045E0900094F0900046E0900095F09E
:1019B500900047E0900096F0900048E0900097F086
:1019C500900033E0900099F0900034E090009AF098
:1019D500900035E090009BF0900036E090009CF080
:1019E5007400900082F0745A900125F074469001BD
:1019F50026F07420900127F07435900128F0744882
:101A0500900129F0745090012AF0743190012BF067
:101A1500743990012CF0742090012DF074359001EB
:101A25002EF0745390012FF07470900130F07465AE
:101A3500900131F07465900132F07464900133F0D7
:101A45009003D4E0900414F0743A90074EF074FDBE
:101A550090074FF012008F900004E4F0A3F090007F
:101A6500067475F0A37430F09000087475F0A374D3
:101A750030F085595AD2CA754C00D29C741B90001F
:101A850023F0E556C394065005E551B55203021BF4
:101A95004DC207E55175F040A4FFAEF09003221248
:101AA500001EE030E003D38001C3B34008E5B54430
:101AB50010F5B58006E5B554EFF5B5E55175F0407F
:101AC500A4FFAEF090032312001EE030E003D380A4
:101AD50001C3B34008E5B54420F5B58006E5B55426
:101AE500DFF5B5E55175F040A4FFAEF09003241283
:101AF500001EE030E003D38001C39287E55175F005
:101B050040A4FFAEF090032512001EE030E003D3A1
:101B15008001C3920CE55175F040A4FFAEF090032F
:101B25002612001EE030E003D38001C3920D8551DB
:101B350052AE29AF2A7405BE00039F5007E545D371
:101B4500940550028002D290E556D39405500302C5
:101B55001D38C207E551D394015003021C29E551F4
:101B650075F040A4FFAEF090031E12001EE0A829F8
:101B7500B80007D3952A40021551E5516552700307
:101B8500021C26E55175F040A4FFAEF09003221229
:101B9500001EE030E003D38001C3B34008E5B5443F
:101BA50010F5B58006E5B554EFF5B5E55175F0408E
:101BB500A4FFAEF090032312001EE030E003D380B3
:101BC50001C3B34008E5B54420F5B58006E5B55435
:101BD500DFF5B5E55175F040A4FFAEF09003241292
:101BE500001EE030E003D38001C39287E55175F014
:101BF50040A4FFAEF090032512001EE030E003D3B1
:101C05008001C3920CE55175F040A4FFAEF090033E
:101C15002612001EE030E003D38001C3920D8551EA
:101C250052021D38E556B406519000ACE030E0088C
:101C3500E5B54410F5B58006E5B554EFF5B590006A
:101C4500ADE030E008E5B54420F5B58006E5B554CE
:101C5500DFF5B59000AEE030E003D38001C3928795
:101C65009000AFE030E003D38001C3920C9000B048
:101C7500E030E003D38001C3920DE556B4075E90D2
:101C850000A5E030E008E5B54410F5B58006E5B5FA
:101C950054EFF5B59000A6E030E008E5B54420F531
:101CA500B58006E5B554DFF5B5AE29AF2A7406BE95
:101CB5000011D39F400D9000A7E030E003D38001D1
:101CC500C392879000A8E030E003D38001C3920C53
:101CD5009000A9E030E003D38001C3920DE556B42E
:101CE500085190009EE030E008E5B54410F5B58058
:101CF50006E5B554EFF5B590009FE030E008E5B591
:101D05004420F5B58006E5B554DFF5B59000A0E0B3
:101D150030E003D38001C392879000A1E030E00357
:101D2500D38001C3920C9000A2E030E003D3800180
:101D3500C3920D900072E06058E54575F00284FF8E
:101D45007E0090014E12001EE0F55DE54775F00A34
:101D550084FF7E0090024E12001EE0F55EE55D25D3
:101D65005ED39464400BE55D255EC39464F55D80A8
:101D750003755D00E55D75F00284FF7E008F5DEF04
:101D8500C394335007EF24CDF55D8003755DFF8067
:101D95001CE54575F00284FF7E0090014E12001E81
:101DA500E075F00284FF7E00EF24CDF55DE595C377
:101DB500955D4004C2938002D293A207B34005E526
:101DC50056B407037574CDE595C395744004C29464
:101DD5008002D294E54575F00284FF7E0090018073
:101DE50012001EE075F00284FF7E00EF24CDF57031
:101DF500E595C395705006A20CB3B340028004D29A
:101E0500918002C291E54575F00284FF7E00900144
:101E1500B212001EE075F00284FF7E00EF24CDF5BE
:101E250071E595C395715006A20DB3B340028004C8
:101E3500D2928002C292E543C394064003022487EE
:101E4500A2EDB35003022487C2EDE5436003021FF0
:101E5500A07E017F00E5BE1241A7E5BD2FFF500121
:101E65000E900000EEF0A3EFF0900029E0B401170A
:101E75007E0F7FFF900000E0FCA3E0FD12000390C1
:101E85000000EEF0A3EFF0900079E0B4025B900063
:101E950000E0FEA3E0FF90000AE0FCA3E0FDEDD327
:101EA5009FEC9E400F900000E0F8A3E090000AC868
:101EB500F0A3C8F0900000E0FEA3E0FF90000CE066
:101EC500FCA3E0FDEFD39DEE9C400F900000E0F8F1
:101ED500A3E090000CC8F0A3C8F0900000E0FEA3BA
:101EE500E0FF74041241998F44900079E07060908E
:101EF5000000E0FEA3E0FF90000AE0FCA3E0FDEF98
:101F0500D39DEE9C400D120003900000EEF0A3EF70
:101F1500F08007900000E4F0A3F0900000E0FEA33D
:101F2500E0FF74101241A7900026E08E048F05FF94
:101F3500124189900000ECF0A3EDF07400D39D747C
:101F4500019C4008900001E0F54480037544FFE5DD
:101F55004475F00AA4FFAEF074198E048F05FF12C4
:101F650041898D45ED2532FFAE3150010E740112C8
:101F750041998F45854532753100EFD39462400311
:101F8500754562900072E064016006900066E0604D
:101F9500028005754301800375BB17E543B4010253
:101FA50080030220907E017F00E5BE1241A7E5BDBA
:101FB5002FFF50010E900000EEF0A3EFF09000729D
:101FC500E0B4017EE53445336025AC33AD341DBD49
:101FD500FF011C8F028E038C068D07903E71120047
:101FE5002EE493FE740193FFEFC39AEE9B400280AB
:101FF5000578331241D1AE33AF3474B3BE0025D367
:102005009F4021900000E0FCA3E0FD0FBF00010E02
:10201500903E7112002EE493FE740193FFEDC39F71
:10202500EC9E40028005783312003FAE33AF34E5B5
:102035006B1241A774648E048F05FF1241898D4789
:102045008033900066E0602D900000E0FEA3E0FF85
:10205500EFD39400EE9408400F900066E0B40104BD
:10206500C2098002D209800D900066E0B40104D255
:10207500098002C209900072E06402600690006661
:10208500E0600575BB168003754302E543B40202A3
:10209500800302217E7E017F00E5BE1241A7E5BDDA
:1020A5002FFF50010E900000EEF0A3EFF0900072AC
:1020B500E0B4027EE53445336025AC33AD341DBD57
:1020C500FF011C8F028E038C068D07903D071200C1
:1020D5002EE493FE740193FFEFC39AEE9B400280BA
:1020E5000578331241D1AE33AF3474B3BE0025D376
:1020F5009F4021900000E0FCA3E0FD0FBF00010E12
:10210500903D0712002EE493FE740193FFEDC39FEB
:10211500EC9E40028005783312003FAE33AF34E5C4
:102125006B1241A774648E048F05FF1241898D4798
:102135008033900066E0602D900000E0FEA3E0FF94
:10214500EFD39400EE9408400F900066E0B40104CC
:10215500C2098002D209800D900066E0B40104D264
:10216500098002C209900072E07003754700900073
:1021750066E07002C20975BB1FE543B403457E01E5
:102185007F00E5BE1241A7E5BD2FFF50010E90006F
:1021950000EEF0A3EFF074091241A774E68E048FE8
:1021A50005FF1241898C418D42E54A2DFD50010CF8
:1021B50074018C068D071241998E418F4285424AE2
:1021C50075BB19E543B40402800302236F7E017FCA
:1021D50000E5BE1241A7E5BD2FFF50010E9000009E
:1021E500EEF0A3EFF074041241998F4BE565B4014D
:1021F5000280030222E2756C00756C00E56CD394D5
:102205000740030222A0E56C9000411241BFE0D3D4
:10221500954B501AE56C9000411241BFE0F404253E
:102225004BFEE56C9000371241BFEEF08017E56C70
:102235009000411241BFE0C3954BFEE56C9000371D
:102245001241BFEEF0E56CC394044009900084E0B0
:10225500C3956C503BE56C6029E56C9000371241E5
:10226500BFFEE0FFEE90003FE0D39F4013E56C908A
:1022750000371241BFE090003FF0E56C900040F060
:10228500800E900037E090003FF07400900040F021
:10229500786C740126F64003022201900040E0F4B8
:1022A500042408F556E556D394054002C290E55836
:1022B50065566029E556B4070CAE29AF2A7405BEEC
:1022C50000059F40028002D287855658E556C39483
:1022D500045007E55604F5578003855657E565D341
:1022E50094014049E54BD3946E4004D2108002C25C
:1022F50010755605E565B40205A210B340028003CA
:10230500755607E565B40306A210B3B34002800312
:10231500755607E55865566014855658E556C394B5
:10232500045007E55604F5578003855657E558656B
:10233500566008E55104F552855658E556B4070828
:10234500E5B54480F5B58006E5B5547FF5B5E556A8
:1023550064066005E556B40808E5B54440F5B58062
:1023650006E5B554BFF5B575BB13E543B405028065
:10237500030224837E017F00E5BE1241A7E5BD2F40
:10238500FF50010E900000EEF0A3EFF0740412412F
:10239500998F46E564B402028003022480756C00BF
:1023A500756C00E56CD394034003022437E56C900B
:1023B50000331241BFE0D39546501AE56C900033C7
:1023C5001241BFE0F4042546FEE56C90002D124154
:1023D500BFEEF08017E56C9000331241BFE0C39566
:1023E50046FEE56C90002D1241BFEEF0E56C6029CC
:1023F500E56C90002D1241BFFEE0FFEE900031E04C
:10240500D39F4013E56C90002D1241BFE090003141
:10241500F0E56C900032F0800E90002DE0900031D8
:10242500F07400900032F0786C740126F6400302D7
:1024350023A8900082E07043E52A45296036E559D6
:10244500C39403500A900032E004C3940340028011
:1024550007900032E004F559E559D39402400A90FB
:102465000032E004D3940250028007900032E00469
:10247500F5598007900032E004F55975BB180543FE
:10248500D2ECE55FD39404500302263F75CF01C219
:1024950093AE35AF367488D39F74139E4005A2A5BD
:1024A500B34014AE35AF367488D39F74139E400580
:1024B500A2A4B340028048783512003FAE35AF364E
:1024C500EFB4883BEEB41337A2A5B3500990004F83
:1024D500E0D395515002800405518011A2A5B35057
:1024E5000890004FE0655160028002D207A2A4B3B4
:1024F5005007E551D39401500280041551C207A23B
:10250500A5B3B35006A2A4B3B34002800675360046
:10251500753500E551655270030225C1E55175F029
:1025250040A4FFAEF090032212001EE030E003D37A
:102535008001C3B34008E5B54410F5B58006E5B59F
:1025450054EFF5B5E55175F040A4FFAEF0900323C7
:1025550012001EE030E003D38001C3B34008E5B5A7
:102565004420F5B58006E5B554DFF5B5E55175F0C0
:1025750040A4FFAEF090032412001EE030E003D328
:102585008001C39287E55175F040A4FFAEF090033A
:102595002512001EE030E003D38001C3920CE55103
:1025A50075F040A4FFAEF090032612001EE030E067
:1025B50003D38001C3920DC294855152A2074005F1
:1025C5007574CD80037574FFE595C395744004C299
:1025D500948002D294E54575F00284FF7E00900157
:1025E5008012001EE075F00284FF7E00EF24CDF519
:1025F50070E595C395705006A20CB3B340028004F4
:10260500D2918002C291E54575F00284FF7E00906B
:1026150001B212001EE075F00284FF7E00EF24CDAA
:10262500F571E595C395715006A20DB3B3400280CF
:1026350004D2928002C292022491A20FB3500DAE31
:1026450025AF2674E8C39F74039E4002800575FF7D
:10265500A0D20FAE25AF26EFD39420EE944E5003B3
:10266500022753120471C28E758D00758B00754C4F
:1026750000D28EC2077573007572007574CD7551E1
:1026850005752400752300755400755B00C296908E
:102695000059E06004D2958002C29590004AE0B4EA
:1026A5000104D2978002C297900049E0B40104D298
:1026B500A08002C2A0A209B34004D2A28002C2A295
:1026C50090006BE06018123826A200B34008E5B50B
:1026D5004408F5B58006E5B554F7F5B58002C200A6
:1026E50090006EE0601812397BA202B34008E5B590
:1026F5004402F5B58006E5B554FDF5B58006E5B5AA
:1027050054FDF5B590000E74FDF0A374E8F0E543B3
:10271500B40603754300900025E4F0752600752581
:1027250000758D00758B00754C00900024E0C394F6
:10273500035008900024E004F08006740390002400
:10274500F0900024E0B40306E5B554FEF5B5AE27D8
:10275500AF28EFD39410EE9427401CC2CA75CD0064
:1027650075CC00752800752700D2CA754E00752AEC
:0A27750000752900755500020AEFF7
:103B2D0000000100013201640196019602000212AB
:103B3D0002240200020003000340038003C00400BE
:103B4D000440048004C005000600060006000600BF
:103B5D00060006000600060000FF01310163019515
:103B6D0001FF01FF0211022302FF02FF02FF033FCB
:103B7D00037F03BF03FF043F047F04BF04FF05FF62
:103B8D0006FF06FF06FF06FF06FF06FF06FF06FF00
:103B9D000FAA0FA50F9F0F9A0F940F8D0F870F80F0
:103BAD000F780F710F680F600F570F4E0F450F3BBA
:103BBD000F300F250F1A0F0E0F020EF50EE80EDB4C
:103BCD000ECC0EBE0EAE0E9F0E8E0E7D0E6C0E5AD0
:103BDD000E470E340E200E0C0DF70DE20DCB0DB56C
:103BED000D9D0D850D6D0D540D3A0D200D050CE936
:103BFD000CCE0CB10C940C760C580C3A0C1B0BFB28
:103C0D000BDB0BBB0B9A0B790B570B350B130AF117
:103C1D000ACE0AAB0A870A640A400A1C09F809D4BD
:103C2D0009B0098C09670943091F08FB08D608B2BA
:103C3D00088E086A0846082307FF07DC07B90796B0
:103C4D0007730751072F070D06EC06CA06AA06894A
:103C5D0006690649062A060A05EC05CD05B005924A
:103C6D0005750558053C0520050504EA04CF04B586
:103C7D00049C04820469045104390422040B03F4E6
:103C8D0003DE03C803B2039D038903750361034D6E
:103C9D00033B03280316030402F202E102D102C022
:103CAD0002B002A00291028202730265025702491C
:103CBD00023C022F02220216020901FD01F201E669
:103CCD0001DB01D001C601BB01B101A7019D01942A
:103CDD00018B018201790170016801600158015069
:103CED000148014101390132012B0125011E011845
:103CFD000111010B010500FF00FA0FA60FA00F998E
:103D0D000F920F8B0F840F7C0F740F6B0F620F5878
:103D1D000F4E0F430F380F2C0F1F0F120F050EF7FD
:103D2D000EE80ED80EC80EB70EA50E930E800E6CB3
:103D3D000E580E420E2C0E150DFD0DE40DCB0DB1D2
:103D4D000D950D790D5D0D3F0D200D010CE10CC094
:103D5D000C9E0C7C0C590C350C100BEA0BC40B9EF5
:103D6D000B760B4F0B260AFD0AD40AAA0A800A55B8
:103D7D000A2A09FF09D409A8097C0950092508F95F
:103D8D0008CD08A10875084A081E07F307C8079D46
:103D9D0007730749072006F706CE06A6067E0657C7
:103DAD000630060A05E405BF059B05770554053267
:103DBD00051004EF04CE04AE048F047104530435D2
:103DCD00041903FD03E203C703AD0394037B0363EF
:103DDD00034B0334031E030802F302DE02CA02B6CC
:103DED0002A30291027F026D025C024C023C022C86
:103DFD00021D020E020001F201E401D701CA01BE4B
:103E0D0001B101A6019A018F0185017A0170016648
:103E1D00015D0153014A014101390131012901219E
:103E2D0001190112010B010400FD00F700F000EA79
:103E3D0000E400DE00D900D300CE00C900C400BFED
:103E4D0000BA00B500B100AD00A800A400A0009C10
:103E5D00009900950091008E008A008700840081F2
:043E6D00007E007B58
:1027A000751A00751900AE19AF1AAC17AD18EDC344
:1027B0009FEC9E401674FF12417975CF01781A7410
:1027C0000126F6500418E436F650DB22900786E422
:1027D000F0A3F0751000750F00751300751400C29A
:1027E00011D21222C2AF75D900758F0375B7A575C6
:1027F000B7F190F800E4F0758F0175B7A575B7F1E2
:10280000E50890F800F075B7A575B7F190F801E408
:10281000F075B7A575B7F190079DE090F802F075D7
:10282000B7A575B7F19007A1E090F803F075B7A5CB
:1028300075B7F190079EE090F804F075B7A575B7ED
:10284000F190079FE090F805F075B7A575B7F19086
:1028500007A0E090F806F075B7A575B7F19007A24C
:10286000E090F807F0758F0075D940D2AF2290073D
:1028700088E0B4AB61C2AF75D90075B62275F52298
:10288000758F0375B7A575B7F1740090F600F075F4
:102890008F01750A00750900AE09AF0A7413BE00F6
:1028A000279F402475B7A575B7F190078912001EC0
:1028B000E0FC90F60012001EECF0780A740126F697
:1028C000500418E436F650D0758F0075F51175B6C2
:1028D0002075D940D2AF22C2AF75D90075F52275E7
:1028E0000A00750900AE09AF0A7413BE00229F40AA
:1028F0001F90F60012001EE493FC90078912001E40
:10290000ECF0780A740126F6500418E436F650D537
:1029100075F51175D940D2AF22900788E0B4AA02AC
:102920008003022A56C2AF75D90075B62275F5220A
:10293000758F0375B7A575B7F1740090EE00F0754B
:10294000B7A575B7F1740090F000F075B7A575B72D
:10295000F1740090F200F075B7A575B7F1740090AE
:10296000F400F0758F01750A00750900AE09AF0A11
:1029700074FFC39F74019E402475B7A575B7F1908D
:10298000004E12001EE0FC90EE0012001EECF078EB
:102990000A740126F6500418E436F650CF750A0082
:1029A000750900AE09AF0A74FFC39F74019E4024ED
:1029B00075B7A575B7F190024E12001EE0FC90F0BD
:1029C0000012001EECF0780A740126F6500418E498
:1029D00036F650CF750A00750900AE09AF0A74FFCC
:1029E000C39F74019E402475B7A575B7F190044E3E
:1029F00012001EE0FC90F20012001EECF0780A7447
:102A00000126F6500418E436F650CF750A00750911
:102A100000AE09AF0A74FFC39F74019E402475B7CE
:102A2000A575B7F190064E12001EE0FC90F400125E
:102A3000001EECF0780A740126F6500418E436F60D
:102A400050CF758F0075F51175B62075D940D2AF8E
:102A5000743A90074EF022900788E0B4AA028003EF
:102A6000022B94C2AF75D90075B62275F522758F09
:102A70000375B7A575B7F1740090E600F075B7A5BA
:102A800075B7F1740090E800F075B7A575B7F174EB
:102A90000090EA00F075B7A575B7F1740090EC00EE
:102AA000F0758F01750A00750900AE09AF0A74FF51
:102AB000C39F74019E402475B7A575B7F190004E71
:102AC00012001EE0FC90E60012001EECF0780A7482
:102AD0000126F6500418E436F650CF750A00750941
:102AE00000AE09AF0A74FFC39F74019E402475B7FE
:102AF000A575B7F190024E12001EE0FC90E800129E
:102B0000001EECF0780A740126F6500418E436F63C
:102B100050CF750A00750900AE09AF0A74FFC39F54
:102B200074019E402475B7A575B7F190044E12004C
:102B30001EE0FC90EA0012001EECF0780A740126F8
:102B4000F6500418E436F650CF750A00750900AE49
:102B500009AF0A74FFC39F74019E402475B7A57521
:102B6000B7F190064E12001EE0FC90EC0012001E21
:102B7000ECF0780A740126F6500418E436F650CFCB
:102B8000758F0075F51175B62075D940D2AF743ABE
:102B900090074EF022900788E0B4AA028003022C2E
:102BA000D2C2AF75D90075B62275F522758F03753F
:102BB000B7A575B7F1740090DE00F075B7A575B7CD
:102BC000F1740090E000F075B7A575B7F17400904E
:102BD000E200F075B7A575B7F1740090E400F075E8
:102BE0008F01750A00750900AE09AF0A74FFC39F13
:102BF00074019E402475B7A575B7F190004E120080
:102C00001EE0FC90DE0012001EECF0780A74012633
:102C1000F6500418E436F650CF750A00750900AE78
:102C200009AF0A74FFC39F74019E402475B7A57550
:102C3000B7F190024E12001EE0FC90E00012001E60
:102C4000ECF0780A740126F6500418E436F650CFFA
:102C5000750A00750900AE09AF0A74FFC39F7401BD
:102C60009E402475B7A575B7F190044E12001EE082
:102C7000FC90E20012001EECF0780A740126F65077
:102C80000418E436F650CF750A00750900AE09AF96
:102C90000A74FFC39F74019E402475B7A575B7F1F0
:102CA00090064E12001EE0FC90E40012001EECF0B4
:102CB000780A740126F6500418E436F650CF758F62
:102CC0000075F51175B62075D940D2AF743A9007EA
:102CD0004EF022900788E0B4AA028003022E10C2B0
:102CE000AF75D90075B62275F522758F0375B7A536
:102CF00075B7F1740090D600F075B7A575B7F1748B
:102D00000090D800F075B7A575B7F1740090DA009F
:102D1000F075B7A575B7F1740090DC00F0758F0100
:102D2000750A00750900AE09AF0A74FFC39F7401EC
:102D30009E402475B7A575B7F190004E12001EE0B5
:102D4000FC90D60012001EECF0780A740126F650B2
:102D50000418E436F650CF750A00750900AE09AFC5
:102D60000A74FFC39F74019E402475B7A575B7F11F
:102D700090024E12001EE0FC90D80012001EECF0F3
:102D8000780A740126F6500418E436F650CF750A16
:102D900000750900AE09AF0A74FFC39F74019E401D
:102DA0002475B7A575B7F190044E12001EE0FC9093
:102DB000DA0012001EECF0780A740126F6500418AE
:102DC000E436F650CF750A00750900AE09AF0A74F3
:102DD000FFC39F74019E402475B7A575B7F1900697
:102DE0004E12001EE0FC90DC0012001EECF0780A8F
:102DF000740126F6500418E436F650CF758F00752E
:102E0000F51175B62075D940D2AF743A90074EF0DF
:102E100022C2AF75D90075F522750A00750900AE9A
:102E200009AF0A74FFC39F74019E401F90EE001209
:102E3000001EE493FC90004E12001EECF0780A7421
:102E40000126F6500418E436F650D4750A007509C8
:102E500000AE09AF0A74FFC39F74019E401F90F03B
:102E60000012001EE493FC90024E12001EECF0785B
:102E70000A740126F6500418E436F650D4750A0098
:102E8000750900AE09AF0A74FFC39F74019E401F0D
:102E900090F20012001EE493FC90044E12001EEC0F
:102EA000F0780A740126F6500418E436F650D4750A
:102EB0000A00750900AE09AF0A74FFC39F74019E32
:102EC000401F90F40012001EE493FC90064E120086
:102ED0001EECF0780A740126F6500418E436F65019
:102EE000D475F51175D940D2AF22C2AF75D900752E
:102EF000F522750A00750900AE09AF0A74FFC39F79
:102F000074019E401F90E60012001EE493FC9000A6
:102F10004E12001EECF0780A740126F6500418E4F4
:102F200036F650D4750A00750900AE09AF0A74FF71
:102F3000C39F74019E401F90E80012001EE493FCA2
:102F400090024E12001EECF0780A740126F650042E
:102F500018E436F650D4750A00750900AE09AF0AB8
:102F600074FFC39F74019E401F90EA0012001EE48C
:102F700093FC90044E12001EECF0780A740126F6C1
:102F8000500418E436F650D4750A00750900AE09ED
:102F9000AF0A74FFC39F74019E401F90EC001200A3
:102FA0001EE493FC90064E12001EECF0780A7401A9
:102FB00026F6500418E436F650D475F51175D9404C
:102FC000D2AF22C2AF75D90075F522750A00750916
:102FD00000AE09AF0A74FFC39F74019E401F90DECC
:102FE0000012001EE493FC90004E12001EECF078DC
:102FF0000A740126F6500418E436F650D4750A0017
:10300000750900AE09AF0A74FFC39F74019E401F8B
:1030100090E00012001EE493FC90024E12001EECA1
:10302000F0780A740126F6500418E436F650D47588
:103030000A00750900AE09AF0A74FFC39F74019EB0
:10304000401F90E20012001EE493FC90044E120018
:103050001EECF0780A740126F6500418E436F65097
:10306000D4750A00750900AE09AF0A74FFC39F74D6
:10307000019E401F90E40012001EE493FC90064E57
:1030800012001EECF0780A740126F6500418E4369B
:10309000F650D475F51175D940D2AF22C2AF75D9AB
:1030A0000075F522750A00750900AE09AF0A74FFB4
:1030B000C39F74019E401F90D60012001EE493FC33
:1030C00090004E12001EECF0780A740126F65004AF
:1030D00018E436F650D4750A00750900AE09AF0A37
:1030E00074FFC39F74019E401F90D80012001EE41D
:1030F00093FC90024E12001EECF0780A740126F642
:10310000500418E436F650D4750A00750900AE096B
:10311000AF0A74FFC39F74019E401F90DA00120033
:103120001EE493FC90044E12001EECF0780A740129
:1031300026F6500418E436F650D4750A00750900D6
:10314000AE09AF0A74FFC39F74019E401F90DC005C
:1031500012001EE493FC90064E12001EECF0780A5A
:10316000740126F6500418E436F650D475F511753E
:10317000D940D2AF22E51464046006E59964FF608B
:10318000028031A2114004D2118027E51460087436
:10319000E62514900023F0E513600874F0251390E1
:1031A0000023F0E514B4010280FE751400751300CD
:1031B000C2118002C211E514903AD0F82828737524
:1031C0001400E599B4FF03751301E599B4FE037586
:1031D0001302E599B4FD03751303E599B4FC037577
:1031E0001304E599B4FA03751305E599B4FB067564
:1031F0001401120471E599B4F906751404120471EE
:10320000E599D394E54007E599C394F04002801610
:103210008599157514027E017F00E515C394E612A9
:1032200041A78E0D8F0E900786E4F0A3F0E599D3A9
:1032300094C44007E599C394E64002802885991517
:1032400075140374E5C39515F50E750D00AE0DAF3D
:103250000E903B2D12002EE493F874019390078694
:10326000C8F0A3C8F0D2990236E4900786E0FEA326
:10327000E0FFEFC39400EE94054009EFD394FFEE16
:1032800094064013900786E0FEA3E0FF90004E12E4
:10329000001EE599F0800385996D90078612000E57
:1032A000900786E0FEA3E0FFEFB40106EEB407024C
:1032B00080030234F490074EE0B43C0280030234F1
:1032C000F4A20AB35005A20BB340030233E7C29C39
:1032D00090007AE090078CF0900057E090078DF016
:1032E000900062E090078EF0900063E090078FF00E
:1032F000900074E0900790F090007CE0900791F0CF
:1033000090007DE0900792F0900080E0900793F0AD
:10331000900081E0900794F090013AE0900795F0DA
:1033200090013BE0900796F090013CE0900797F009
:10333000900090E0900798F0900091E0900799F04D
:10334000900092E090079AF0900093E090079BF035
:10335000900094E090079CF0900095E090079DF01D
:10336000900096E090079EF0900097E090079FF005
:10337000900099E09007A0F090009AE09007A1F0EB
:1033800090009BE09007A2F090009CE09007A3F0D3
:103390007400900082F012008F74AB900788F012D6
:0A33A000286E74AA900788F0E55922
:063AD0000231BF02326A60
:1033AA00903AF1F82828738012122919800D122AEE
:0B33BA00578008122B958003122CD3C3
:0F3AF1000233B10233B30233B80233BD0233C222
:1033C500900788E4F090013AE0700C90013BE070C2
:1033D5000690013CE060028004C20A8002D20A0223
:1033E50034E9C29C900078E0900789F090005EE097
:1033F50090078AF090005FE090078BF090007AE0EC
:1034050090078CF0900057E090078DF0900062E0F7
:1034150090078EF0900063E090078FF0900074E0C5
:10342500900790F090007CE0900791F090007DE08F
:10343500900792F0900080E0900793F0900081E073
:10344500900794F090013AE0900795F090013BE0E9
:10345500900796F090013CE0900797F0900090E07F
:10346500900798F0900091E0900799F0900092E015
:1034750090079AF0900093E090079BF0900094E0FD
:1034850090079CF0900095E090079DF0900096E0E5
:1034950090079EF0900097E090079FF0900099E0CC
:1034A5009007A0F090009AE09007A1F090009BE0B3
:1034B5009007A2F090009CE09007A3F074009000A4
:1034C50082F074AB900788F012286E74AA90078872
:1034D500F0122919122A57122B95122CD3D29C754A
:1034E50099FB80FED29C7514007513007599FB023B
:1034F50036E4900786E0FEA3E0FFEF4E700685995F
:1035050010750F00900786E0FEA3E0FF74016F4E73
:10351500701BAC0FAD10AA0DAB0EED2BFBEC3AFA00
:103525008A068B0790004E12001EE599F0900786DB
:1035350012000E900786E0FEA3E0FF74026F4E7046
:103545000C12008F8515997514007513000236E469
:10355500900786E0FEA3E0FF90004E12001EE5995D
:10356500F090078612000E900786E0FEA3E0FFAC00
:103575000DAD0E8F028E038C068D07903B651200F4
:103585002EE493F9740193FEEAD39EEB99400985E5
:1035950015997514007513000236E4900786E0FE50
:1035A500A3E0FF90004E12001EE599F090078612E9
:1035B500000E900786E0FEA3E0FFEFB40006EEB430
:1035C500010280030236E490001CE0D394C7400B4F
:1035D50090001CE0C394C8F516801A90001CE0D337
:1035E5009463400B90001CE0C39464F5168006902C
:1035F500001CE0F516E51675F002A4FFAEF08F6C21
:10360500EF90004E1241BFEFFCE0FDEC900051122F
:1036150041BFEDFCE0FDEC2DB5160280030236D668
:103625000FEF90004E1241BFE56CFFE0FCEF9000FC
:10363500521241BFECFFE0FCEFC39CB516028003BC
:103645000236D6E56C9000501241BFE56CFFE0FCF8
:10365500EF9000531241BFECFFE0FCEF2CB5167163
:10366500E56C9000541241BFE0C3951690079DF09C
:10367500E56C9000551241BFE0C3951690079EF08A
:10368500E56C9000581241BFE0C3951690079FF076
:10369500E56C9000591241BFE0C395169007A0F064
:1036A500E56C90005A1241BFE0C395169007A1F052
:1036B500E56C90005B1241BFE0C395169007A2F040
:1036C5001227E47599F97518647517001227A080FB
:0F36D500FE7599FF7518647517001227A080FE07
:093AD6000234F70235550235A057
:1036E40022E513903ADFF8282873023825900786DC
:1036F400E0FEA3E0FF90001212001EE0F59990078F
:103704008612000E900786E0FEA3E0FF74116F4E50
:1037140070037513000238258563990238259007D4
:1037240086E0FEA3E0FF90004E12001EE0F599EF44
:10373400B40107EEB4070375130090078612000E58
:07374400023825900787E021
:0F3ADF000236EE0236F102371C02372202374759
:10374B00903B00F828287385249902381A852A990A
:10375B0002381A85449902381A85479902381A8516
:10376B00519902381A85619902381A85569902388F
:10377B001A85599902381A756F00900069E0700626
:10378B00900068E060028016A2A44006E56F440436
:10379B00F56FA2A54006E56F4402F56F801A900005
:1037AB004AE0B40106E56F4410F56F900049E0B4B0
:1037BB000106E56F4420F56FA207B34006E56F44A1
:1037CB0001F56FA209B34006E56F4408F56F856FED
:1037DB0099803CA212B340077599FAC2128017A2C6
:1037EB000EB3400575990F800B900023E0F599906F
:1037FB000023E4F0C20E80178542998012854B9905
:0F380B00800D85469980087599FC800375130020
:103B000002375202375802375E02376402376A02C0
:103B1000377002377602377C0237820237DE02388E
:0D3B20000302380802380D0238120238176F
:0B381A0090078612000E800312004889
:033AEE0002382279
:103825002290006BE0B4010385241190006BE0B495
:103835000203852A1190006BE0B4030385441190BF
:10384500006BE0B4040385471190006BE0B40503F9
:1038550085511190006BE0B4060385561190006BFD
:10386500E0B4070385591190006CE0FE90006DE00F
:10387500C39E50030238FC90006BE0D39404402CA7
:1038850090006CE0D39511500990006DE0C395113F
:1038950050028002D20090006CE0D395115009903F
:1038A500006DE0C395115002C200804990006BE0A5
:1038B500B4041890006DE0C395115002D200900039
:1038C5006CE0D395114002C200802A90006CE0C3E1
:1038D5009511500990006DE0D3951150028002D2E8
:1038E5000090006CE0D39511500990006DE0C395F0
:1038F500115002C200807E90006BE0D39404402CEE
:1039050090006CE0C39511400990006DE0D39511CE
:1039150040028002C20090006CE0C39511400990FE
:10392500006DE0D395114002D200804990006BE014
:10393500B4041890006CE0C395115002C2009000C9
:103945006DE0D395114002D200802A90006CE0C34F
:103955009511400990006DE0D395114002D2009079
:10396500006CE0D39511400990006DE0C3951140BE
:10397500028002C2002290006EE0B401038524118A
:1039850090006EE0B40203852A1190006EE0B40346
:103995000385441190006EE0B4040385471190003F
:1039A5006EE0B4050385511190006EE0B406038501
:1039B500561190006EE0B4070385591190006FE031
:1039C500FE900070E0C39E5003023A5190006EE0F5
:1039D500D39404402C90006FE0D3951150099000CA
:1039E50070E0C3951150028002D20290006FE0D3BF
:1039F50095115009900070E0C395115002C20280E4
:103A05004990006EE0B40418900070E0C395115021
:103A150002D20290006FE0D395114002C202802AC3
:103A250090006FE0C395115009900070E0D3951197
:103A350050028002D20290006FE0D3951150099098
:103A45000070E0C395115002C202807E90006EE0C6
:103A5500D39404402C90006FE0C395114009900069
:103A650070E0D3951140028002C20290006FE0C35E
:103A750095114009900070E0D395114002D2028063
:103A85004990006EE0B4041890006FE0C3951150A2
:103A950002C202900070E0D395114002D202802A42
:103AA50090006FE0C395114009900070E0D3951127
:103AB5004002D20290006FE0D3951140099000704A
:0B3AC500E0C3951140028002C2022203
:0941BF002582F5825002058322DD
:10002E00EF2F500205832582F582E5833E2EF58360
:01003E00229F
:08000300C3EF9DFFEE9CFE22FD
:08003F000806B60002180622B3
:0D000E00A3E004F070061241B5E004F022FA
:0841D1000816B6FF02181622C1
:0E419900048007C3CE13CECF13CFD5E0F6229D
:10404700BC000FBE0008ED8FF084FFADF022E4FE48
:10405700FF22BE000DEF60FE54F0606F20E7030201
:1040670040FDEAC0E0EBC0E078017A0075F001EEB0
:1040770020E710EF25E0FFEE33FE0AC5F023C5F079
:1040870030E7F0EA5407F9096A7A007B0060010813
:10409700C3EC9E40167004ED9F4010ED9FFDEC9E13
:1040A700FCE5F0CA4ACA03F5F08005E5F003F5F030
:1040B700C3EE13FEEF13FFD9D77908CACBCAD8D0FE
:1040C700EAFEEBFFD0E0FBD0E0FA22EC8FF084FCB5
:1040D700ED54F045F0C48FF084FEEDC454F045F084
:1040E700C48FF084FDEEC4FE54F02DFFEE540F3C58
:1040F700FEADF07C0022790078008FF0EC7E08207E
:10410700E70DC3CD33CD33C933C9C833C8DEF08417
:1041170049F9E5F08FF0BE00E6FD7C00E9FFE8FE17
:014127002275
:0E41A700F88FF0A4FFE5F0CE88F0A42EFE22E3
:10417900600D782B024183007830D8FED5E0F82213
:10418900EEC0E07E00124047EFFDEEFCD0E0FE22DB
:03000B0002412887
:03001B000241435C
:03002B0002415E31
:030000000241C8F2
:0941C80075817575D00002065BDB
:0B001E00E5822FF582E5833EF583228A
:0A41B5000582D582021583158222CF
:10412800C0E0C0F0C083C082C0D075D00012065075
:10413800D0D0D082D083D0F0D0E032C0E0C0F0C080
:1041480083C082C0D075D000120653D0D0D082D0A0
:1041580083D0F0D0E032C0E0C0F0C083C082C0D0CD
:1041680075D000120656D0D0D082D083D0F0D0E0DF
:014178003214
:00000001FF
